:020000040000FA
:1000000038040020692600007126000073260000D5
:1000100000000000000000000000000000000000E0
:100020000000000000000000000000007526000035
:100030000000000000000000772600007926000084
:100040007B2600007B2600007B2600007B2600002C
:100050007B2600007B2600007B2600007B2600001C
:100060007B2600007B2600007B2600007B2600000C
:100070007B2600007B2600007B2600007B260000FC
:100080007B2600007B2600007B2600007B260000EC
:100090007B2600007B2600007B2600007B260000DC
:1000A0007B260000D50000007B2600007B26000098
:1000B0007B2600007B2600007B2600007B260000BC
:1000C0000348854602F010FD00480047D7000000B5
:1000D00038040020704700BF00BF00BF59202D49E1
:1000E000086016200860882008600846006800281C
:1000F000F4D000BF00F06BF800BF00202549086075
:1001000000BF382000F01AFC00F0A9FB00F0B7FB9C
:10011000214840680721090608431F49486000F04C
:10012000BAFA0221002000F008FB0321022000F0AF
:1001300004FB0421084600F000FB00F001FA00F087
:10014000F3FB164800F0D8FB1549087800F0F6FBE1
:1001500014490D68E90F49194910134A88181149C3
:10016000096802F08FFA441E2146002000F03AFA96
:100170002146022000F036FA2146042000F032FA2F
:100180000AA000F055FC03E002F068FE02F052FD08
:10019000FAE70000000100500000044020A1070021
:1001A000080000200000002000A24A040D0A4F4B66
:1001B0002000000000BF5920F9490860162008609F
:1001C00088200860084600680028F4D0704710B501
:1001D000042001F0A1FD102001F0FEFB002107200A
:1001E00001F00AFC012001F097FD012001F0F4FB71
:1001F000EC4801F0E1FC042001F0EEFBEA4801F0DC
:1002000097FD00221146E84801F01EFDE74801F085
:100210008FFD032252040C21E44801F015FDE4484F
:1002200001F086FDE34801F083FDE34801F080FD25
:10023000002201214902E04801F006FDDF4801F0FB
:1002400077FD002201214903DC4801F0FDFCDC4878
:1002500001F06EFD002201214904D94801F0F4FCAF
:10026000D84801F065FD002201210907D04801F0BE
:10027000EBFC002201214907CE4801F0E5FCD24801
:1002800001F0F6FAD048401C01F0F2FA0520000710
:10029000406B000A00020521090748630846406BCD
:1002A000332108430521090748630846806B000E87
:1002B000000688630846806BC44908430521090786
:1002C0008863B748C038806800090001B449C03964
:1002D00088600846806805210843B149C0398860B4
:1002E000084680680F2109038843AD49C0398860FA
:1002F0000846806809140843A949C039886000226B
:100300004021B34802F0F8F8A548C0380068000959
:100310000001A349C0390860084600680621084367
:100320009F49C039086008460068F02188439C490D
:10033000C039086008460068602108439849C03900
:100340000860084600680F21090288439449C039B3
:100350000860084600680321490208439049C039F3
:100360000860084600680F21090388438C49C0399A
:100370000860084600680321490308438849C039DA
:100380000860084600680F21090488438449C03981
:100390000860084600680321490408438049C039C1
:1003A0000860084600680F21090588437C49C03968
:1003B0000860084600680321490508437849C039A8
:1003C0000860084600680F21090688437449C0394F
:1003D0000860084600680321490608437049C0398F
:1003E000086005200007C06B0F2109048843052120
:1003F0000907C8630846C06B032149040843052167
:100400000907C8630846006B0F21090388430521CB
:10041000090708630846006B0321490308430521C7
:10042000090708630846006B0F210902884305216C
:10043000090708630846006B0321490208430521A8
:10044000090708630846006BF02188430521090766
:1004500008630846006B602108430521090708630B
:100460000846006B0009000108630846006B06217E
:1004700008430521090708630322102154488030EE
:1004800002F03AF8032220215148803002F034F87B
:10049000032240214E48803002F02EF803228021B2
:1004A0004B48803002F028F803220421484880306D
:1004B00002F022F803220121C902454802F01CF88B
:1004C0000322FF2101314248803002F015F8032257
:1004D000012149023E48803002F00EF8032201213A
:1004E00089023B48803002F007F803220121C9024B
:1004F0003748803002F000F8032201210903344814
:10050000803001F0F9FF0322012149033048803097
:1005100001F0F2FF0322012189032D48803001F010
:10052000EBFF03220121C9032948803001F0E4FFD9
:100530000322012149022648403001F0DDFF10BDB1
:1005400010B5244800680121084322490860224B65
:100550000C2200211F48803800F0EEFB01201D49CD
:100560000861084600680121C9020843194908606A
:1005700010BD10B5062807D2184B84001A51174B2E
:1005800020338400195109E00C2807D2801F144B36
:1005900084001A51124B20338400195110BD000001
:1005A0000001005000A24A04113D80571CFE235652
:1005B0001400C0531500D0530200805E0300C05EDB
:1005C0000400005F1E00004014000004111111001F
:1005D0004040005080000E403F400000300004408A
:1005E0003000144006280FD240084000FA4A830029
:1005F000D150431C9B00D1504908F74A2032830058
:10060000D150431C9B00D150704706280FD24008A0
:100610004000F24A8300D150431C9B00D15049084E
:10062000EE4A20328300D150431C9B00D1507047CA
:1006300010B500234A0894000246143213514B00AF
:1006400003229A4001231B048B401A4343689343BF
:100650004360E34B8C0002463032135100238C0080
:1006600020321351B02212584C00DE4BA3409A4363
:100670004C000223A3401A43B0231A50B42212584C
:100680004C00D84BA3409A434C000123A3401A438B
:10069000B4231A5010BD10B50021CF483038FFF7F1
:1006A000C7FF0121CC483038FFF7C2FF0221CA48FA
:1006B0003038FFF7BDFF0321C7483038FFF7B8FFD8
:1006C0000421C5483038FFF7B3FF0521C248303850
:1006D000FFF7AEFF3F21C048303800F03DFE3F211C
:1006E000BD48303800F0F0FC0021BC483038FFF73E
:1006F0009FFF0121B9483038FFF79AFF0221B74820
:100700003038FFF795FF0321B4483038FFF790FFEA
:100710000421B2483038FFF78BFF0521AF4830384D
:10072000FFF786FF3F21AD48303800F015FE3F212E
:10073000AA48303800F0C8FC10BD70B505460C461C
:10074000FFF738FDA848844200D904462B0002F088
:1007500086FC060405161726273600BF9E48103073
:10076000006B01210906884340189B49103108633A
:10077000224600219848303800F020FE1FE000BFDC
:1007800095483038406F0121090688434118924846
:10079000303841672246022100F010FE0FE000BF12
:1007A0008D483038806F01210906884341188A48F6
:1007B000303881672246042100F000FE00BF00BFF0
:1007C00000BF00208949086000BF70BD70B50546B4
:1007D0000C46FFF7EFFC8448844200D904462B0006
:1007E00002F03DFC060405161726273600BF7B489D
:1007F0001030006B012109068843401877491031F9
:100800000863224600217548303800F0D7FD1FE00C
:1008100000BF72483038406F0121090688434118F3
:100820006E48303841672246022100F0C7FD0FE0D4
:1008300000BF6A483038806F01210906884341189B
:100840006648303881672246042100F0B7FD00BFBA
:1008500000BF00BF00206549086000BF70BD10B533
:1008600064220021624801F05BFD61480068000AD3
:10087000000247305E4908605E48486010BD10B510
:1008800064220121C9065C4801F04AFD5A4800F083
:100890003BFA10BD10B5594A0121C906584801F06C
:1008A0003FFD00BF564800680121490708435449ED
:1008B000086000BF084600F027FA0021192000F068
:1008C000ECF90A20012181404E4A116000BF10BDA1
:1008D00010B54D4A0121C9064C4801F021FD4B4895
:1008E0000068000A000247304849086048484860EC
:1008F000084600F009FA10BD70B5054600240CE06A
:1009000000BF3D488068C007C00F002805D000BF69
:1009100001203949886000BF641C3E49284601F027
:10092000C7FEA042ECDC70BD10B53B4800F0A0FF54
:10093000E1214902394801F043FB10BD014620394D
:10094000374A505CC107C90F002903D00021354A3E
:10095000116202E00121334A1162022101400029A3
:1009600003D000212F4A516202E001212D4A516239
:1009700004210140002903D000212A4A916202E0AB
:100980000121284A916208210140002903D0002159
:10099000244AD16202E00121224AD16210210140A1
:1009A000002903D000211F4A116302E001211D4AE2
:1009B000116320210140002903D00021194A51630D
:1009C00002E00121174A51634021014000292BD048
:1009D0000021144A91632AE03000044030001440A2
:1009E00000A24A0403000300FF0F000000010050B2
:1009F00000000140CB2B00000001014085450100B3
:100A00000000114000E100E040420F0000011140F1
:100A1000FFFFFF0010270000110000040000154038
:100A20005A390000C04200500121BA4A9163704710
:100A30000FB410B5A2B025A80190802102A8019B97
:100A4000249A02F0DFFA04460020019000BF0DE076
:100A500000BFB14989690122D2051140C90D0029A1
:100A6000F7D102A9095CAC4A1160401CA042EFDB3F
:100A700022B010BC08BC04B0184710B502460B46A3
:100A8000D7E0A5480068C1B20D2901D00A2914D1C8
:100A9000A248006804280CDB0020A04C2060A0487D
:100AA0004078303810609F48006818609C48007893
:100AB00010BD0020994C2060BAE0202904D100200C
:100AC000964C20602020F3E7612901D0412904D110
:100AD0000020924C20606120EAE7772901D0572955
:100AE00004D100208D4C20607720E1E7642901D0FB
:100AF000442904D10020894C20606420D8E778295B
:100B000001D0582904D10020844C20607820CFE700
:100B1000462903D0542901D0562905D180480170B7
:100B200001207E4C206083E07C48006801287FDB48
:100B30007D487A4C2468005D6E2826D1302901DB7F
:100B4000392903DD0020754C206071E0754800688C
:100B50000A24604340183038724C206070486F4C53
:100B6000246801556D480068401C6C4C20600628C4
:100B70005ED3002020606A484078303810606948B1
:100B8000006818606648007892E76748634C2468FC
:100B9000005D6D2830D13F290BD100205F4C2060D3
:100BA0005F484078303810605D480078202420434A
:100BB0007EE7302901DB392903DD0020574C206016
:100BC00036E008463038574C20605548534C24686E
:100BD000015552480068401C504C2060062827D31D
:100BE000002020604E484078303810604D48006842
:100BF00018604B4800785BE74B48484C2468005D20
:100C0000884212D145480068401C444C20600628A8
:100C10000ED30020206042484078303810604148B0
:100C2000006818603E48007842E700203B4C206096
:100C300000BF39488069012189030840002800D19C
:100C40001FE7002034E710B500231A46012137487A
:100C500001F084FC35484068C0218843334948602E
:100C60000846406807214903884340182F494860D7
:100C7000084640680121090308432C49486008469A
:100C800040680321090288432849486008464068B3
:100C9000022108432549486010BD10B5002819DA23
:100CA000234A03071B0F083B9B089B00D25883076E
:100CB000DC0EFF23A3409A438B071B0E8407E40E30
:100CC000A3401A431A4B0407240F083CA408A400AD
:100CD0001A5118E0174A03231B02D21883089B00FD
:100CE000D2588307DC0EFF23A3409A438B071B0EC9
:100CF0008407E40EA3401A430E4B032424021B195D
:100D00008408A4001A5110BD016801229207114302
:100D100001607047C04200500000154018000020DC
:100D2000100000200C000020B539000000000D402C
:100D30001CED00E000E100E030B580242458494D6E
:100D40002C400C43144380252C50842424588425A3
:100D50002B5030BD05210907C96801221207114334
:100D600005221207D1601146C9680122120791437A
:100D700005221207D160704710B500290CD18023DD
:100D80001B58FF24F134A3430B431343FF240134C6
:100D90002343802423501EE010290AD180231B58AE
:100DA000FF24F134A3430B430C012343802423503D
:100DB00011E09C231B581B0A1B0213439C24235045
:100DC00080231B58FF24F134A3430B43FF24013439
:100DD00023438024235010BD80210958FF22F13283
:100DE0009143802211507047CA07D20F002A05D0C4
:100DF0008022125802231A4380231A5002220A40EA
:100E0000002A05D08822125802231A4388231A5038
:100E100004220A40002A05D08C22125802231A43C9
:100E20008C231A507047CA07D20F002A05D080229F
:100E3000125802239A4380231A5002220A40002AA1
:100E400005D08822125802239A4388231A5004227C
:100E50000A40002A05D08C22125802239A438C2380
:100E60001A507047F3FBFFFFFEB500200290FBA075
:100E700000680090FA48046A00132040002801D05E
:100E80000020FEBD0120C0042040002801D0F54D07
:100E900000E0F54D012040042040002801D0284604
:100EA000EFE7032080032040800B69460A5C019233
:100EB000E005C00D861C1F2040022040400A871C10
:100EC000019A7A431146AA087243104601F0DAFBF0
:100ED000800002900298D4E7FFB583B004460D4627
:100EE0000127E2480090E248844205D1DC4840698D
:100EF000A1020840029005E0D94840690121490754
:100F0000084002900298002803D1FFF7ADFF064683
:100F10000BE001F037FBD648844203D100F036FDE8
:100F2000064602E000F042FD06467D21C90030463B
:100F300001F0A8FB064601271AE0CE49794308468E
:100F4000314601F09FFB01900599019888420DD22E
:100F500001200003874200D10EE0781CC5494143BF
:100F600001987043814200D806E000E004E07F1C55
:100F7000012000038742E0D900BF781E07466908B8
:100F80008A0021461431885060686A00032191402C
:100F900088436A0001219140084360606068012134
:100FA0000904A94088436060AA00214630310098B6
:100FB0008850019807B0F0BDFFB585B004460D46D6
:100FC0000126AA480290AA48844205D1A448406953
:100FD000A1020840049005E0A148406901214907A9
:100FE000084004900498002803D1FFF73DFF07460E
:100FF0000BE001F0C7FA9E48844203D100F0C6FC22
:10100000074602E000F0D2FC0746012612E038460F
:10101000079901F037FB3146019001F033FB039053
:10102000012109040398884200D902E00398029044
:1010300003E0761C90488642E9D300BF02987043D3
:101040000146384601F01EFB0390701E06466908F3
:101050008A0021461431885069000320884001210C
:101060000904A94008436168814361600298401EF9
:10107000AA002146303102908850029A521C0899E9
:1010800051430846642101F0FDFAAA00214650317F
:101090008850B02000596A007849914088436A001E
:1010A000022191400843B0210851B42000596A0040
:1010B0007249914088436A00012191400843B4215C
:1010C0000851039809B0F0BD026A0A4302627047F2
:1010D00030B5024600200AE0012383400B40002B7C
:1010E00004D000248500134630335C51401C062890
:1010F000F2D330BD026A8A430262704730B50429D8
:1011000011D2F8231C58CD000F23AB409C43F82389
:101110001C5080231343CC00A340F82424582343BD
:10112000F824235012E0FC231B580C1FE5000F2469
:10113000AC40A343FC242350802313430C1FE40042
:10114000A340FC2424582343FC24235030BD10B575
:10115000042908D2F8221258CC008023A3409A43D5
:10116000F8231A5008E0FC2212580B1FDC008023E1
:10117000A3409A43FC231A5010BD10B501231B0451
:101180008B40FF242134235010BD0246FF20213024
:10119000805801231B048B401840002801D00120F7
:1011A00070470020FCE7F0B504460020B6E00125BA
:1011B00085400D40002D2FD0812B0CD0822B0AD0E2
:1011C000882B08D02E4DAB4205D06D1CAB4202D00F
:1011D000AD1DAB4215D14508AE002546C835AD5909
:1011E000274E7F361E4035434608B6002746C8378F
:1011F000BD51C4252D591E07360F3543C426355120
:101200000AE04508AE002546C835AD591D434608DD
:10121000B6002746C837BD51012585401540002D31
:1012200048D0C507ED0F002D2CD14508AE0025464E
:10123000C835AD5903263604B5434608B6002746DF
:10124000C837BD514508AE003D46AD5903263604AA
:1012500035434608B600BD515FE0000001020204BC
:101260000002005000805101001BB700FFFF00008A
:101270000000044040420F00FF0F00000300030085
:10128000018000004508AE002546C835AD5903264B
:10129000B604B5434608B6002746C837BD514508D1
:1012A000AE003D46AD590326B60435434608B600A8
:1012B000BD5132E0C507ED0F002D17D14508AE0036
:1012C0002546C835AD5903263604B5434608B60051
:1012D0002746C837BD514508AE003D46AD590126E9
:1012E000760435434608B600BD5116E04508AE0009
:1012F0002546C835AD590326B604B5434608B600A1
:101300002746C837BD514508AE003D46AD590126B8
:10131000F60435434608B600BD51401C062800D2ED
:1013200045E7F0BD0122520212580A4301235B0235
:101330001A501A1D12580A431B1D1A5070470122D9
:10134000520212588A4301235B021A501A1D125886
:101350008A431B1D1A507047D82212580A43D823BB
:101360001A507047D82212588A43D8231A5070470F
:10137000F0B5CC07E40F8F25AD002D584E08F700CF
:101380001E26BE40B5432601D7003E431E4301271B
:101390003E434F08FF00BE4035438F26B600355010
:1013A000F0BD10B58F22920012584B08DC000123CB
:1013B000A3409A438F239B001A5010BD30B54B08B1
:1013C0009C00034670331B591C0B24034B089D00E3
:1013D000034670335C514B089C00034670331B5925
:1013E00001242404144323434C08A500044670340C
:1013F000635130BD10B54A08930002467032D2588E
:1014000001231B049A434B089C00034670331A5176
:1014100010BD10B525231B011B5814468C402343D7
:1014200025242401235010BD10B525231B011B5872
:1014300014468C40A34325242401235010BD10B52D
:1014400013468B409524A400235010BD10B50246CE
:10145000952080008058FF2301338B4018400028DE
:1014600001D0012000E00020400095239B009B5804
:1014700001248C402340002B01D0012300E00023F5
:10148000184310BD10B5E0231B5814468C4023436D
:10149000E024235010BDE0221258DE4B8B409A43CB
:1014A000E0231A507047DB4A8A40E8231A507047FD
:1014B0000246E8208058D74B8B401840002801D0C6
:1014C000012070470020FCE7E422125807238B40DC
:1014D0001A43E4231A507047E422125807238B4022
:1014E0009A43E4231A5070473F228A40EC231A5053
:1014F00070470246EC2080583F238B40184000285C
:1015000001D0012070470020FCE710B5E0231B58F4
:10151000FF2401348C402343E024235010BDE022FB
:101520001258FF2301338B409A43E0231A5070472F
:10153000FF2201328A40E8231A5070470246E82011
:101540008058FF2301338B401840002801D0012030
:1015500070470020FCE7E022125801238B401A4319
:10156000E0231A507047E022125801238B409A431F
:10157000E0231A50704701228A40E8231A5070472E
:101580000246E820805801238B401840002801D0F3
:10159000012070470020FCE770B5F02424584D0866
:1015A000EE007F25B540AC431D0180263543154331
:1015B0004E08F600B5402C43F0252C5070BD10B5F8
:1015C000F02212584B08DC008023A3409A43F023FA
:1015D0001A5010BD10B5E02212584B08DC008023D1
:1015E000A3401A43E0231A5010BD10B5E022125850
:1015F0004B08DC008023A3409A43E0231A5010BD1F
:101600004A08D30080229A40E8231A50704710B548
:101610000246E82080584B08DC008023A340184095
:10162000002801D0012010BD0020FCE74B08FF225C
:1016300002329A4003231B02C318DA64704710B5C4
:101640000246032000021018C06C4C08FF2302332E
:10165000A3401840002801D0012010BD0020FCE765
:1016600010B5036814468C402343036010BD10B5C9
:10167000036814468C40A343036010BDF0B5059C7D
:1016800049084E0003252D02B540012636068E403E
:101690002E438568B5431E068E40354316024F0023
:1016A000BE40354385608D00064680367451F0BDDE
:1016B00030B5024600200BE0012383400B40002B95
:1016C00005D0936845080124AC4023439360401C37
:1016D0000628F1D330BD30B5024600200BE00123CF
:1016E00083400B40002B05D0946845080123AB4094
:1016F0009C439460401C0628F1D330BD30B50B05E7
:1017000054042343012424041B1984683F256D04D9
:10171000AC432343836030BD8168012212049143AE
:101720008160704781680122D20511438160704752
:1017300081680122D20591438160704730B5036909
:101740004C08E5000724AC40A3434C08E5001446D0
:10175000AC402343036130BD70B5C0242458CE0093
:101760007E25B540AC4315015E0035436D1CCE00AF
:10177000B5402C43C0252C5070BD10B5C022125866
:10178000CC000123A3409A43C0231A5010BD10B5CA
:10179000C0221258CC008023A3401A43C0231A5001
:1017A00010BD10B5C0221258CC008023A3409A432C
:1017B000C0231A5010BD30B5C0231B58CD000124E2
:1017C0002404AC40A343CC0010341546A5402B4361
:1017D000C024235030BD70B5049C15460D432543ED
:1017E000FF26193635505D1E361D355070BD024638
:1017F000FF202130805801238B401840002801D061
:10180000012070470020FCE701228A40FF2321339A
:101810001A50704700000101052109074860704710
:101820000520000780694021084080097047052095
:101830000007406870472B480068C007C00F0121AF
:1018400048407047052000070068704705200007E2
:101850008068012108430521090788607047052039
:101860000007806802210843052109078860704746
:10187000010E05221207891889680122824011434E
:10188000020E05231B07D2189160010E1A46891813
:101890008A68012181408A43010EC9188A60704715
:1018A00005221207926901231A4305231B079A6137
:1018B0001A46926908239A43024305231B079A613B
:1018C0001A46926906239A430A4305231B079A6125
:1018D000704705200007806940084000052109077E
:1018E0008861704700010050F648806840218843B5
:1018F000F4498860704710B510230B43540123430B
:10190000F04C636223469B6840242343ED4CA36064
:101910002346DB691C24A3430343EA4CE36110BD67
:10192000E948006904210843E7490861E54800687F
:1019300080210843E349086030BF7047E2480069EE
:1019400004218843E0490861DE480068802188431B
:10195000DC49086030BF7047DA480068C007C00F34
:10196000002801D0D94870470020FCE7D54800681E
:1019700002210840002801D0880370470020FCE7BE
:1019800010B500F0FFFDD248006810BD10B500F0A2
:10199000F9FDCC48006940210840002803D0CC481C
:1019A0000068400810BDCA480068FBE710B500F0A9
:1019B000E9FDC448006980210840002803D0C448DC
:1019C0000068400810BDC2480068FBE710B500F091
:1019D000D9FDBF48006810BD0146BE4A05E010466B
:1019E000521E002801DC00207047B648C06808403D
:1019F0008842F4D10120F7E770B504460D46B1489E
:101A0000C068102108400646AE480068042108431B
:101A1000AC4908601020FFF7DFFFAA480069C00842
:101A2000C000C01DA749086108468069000900017F
:101A30002843886108460069C008C0002043086147
:101A400000F0A0FD002E05D19E48006804218843C7
:101A50009C49086070BD9B48006A01210904084345
:101A6000984908627047F3B589B00C46FFF7F3FF59
:101A7000099800280ED19348006801210843914934
:101A800008600120FFF7A8FF002006908F4808900B
:101A900002250EE08B48006804210843894908604C
:101AA0001020FFF799FF0120C00406908A48089093
:101AB00004258A48844204D84010844201D9002772
:101AC00012E08748844205D84010844202D9012799
:101AD000640009E08348844205D84010844202D360
:101AE0000327A40000E057E00020C043039000203B
:101AF0000190029034E02946089800F0C3FD05905B
:101B00007949059888422AD978490598884226D289
:101B1000022007901EE0059E07994E4370488642BA
:101B200015D34000864212D8A64201D9301B00E0EE
:101B3000A01B049003990498884208D2049803904B
:101B40000195079802900398002800D106E00798B5
:101B5000401C0790664907988842DCD900BF6D1C7D
:101B6000212DC8D9B803069908430199891E490255
:101B700008430299891E0843524908620420FFF76E
:101B80002BFF781C019A50430146089800F07AFD1B
:101B9000029948430BB0F0BD0998002803D155487D
:101BA0004849086202E05448464908620420FFF7A9
:101BB00013FF00F019F9EDE770B504464148C0681D
:101BC0001021084005464D48844200D904464C483F
:101BD000844200D204463B48006804210843394946
:101BE00008601020FFF7F8FE364800690721084317
:101BF0003449086108468069000900018861084687
:101C0000C068C007C00F002805D061000020FFF7A2
:101C10002AFF04460AE061000120C004FFF723FF09
:101C200004462848C06810210840054601210220CA
:101C3000FFF7E2FE002D05D1224800680421884309
:101C400020490860600870BDF7B586B00022002307
:101C50002C4C2546E0CDE468049703960295059444
:101C6000284D103530CD019500948403240E002CAE
:101C700011D00403A40FA4006D462C59114D183542
:101C800063198403250E8405E40EA5401C68AC434B
:101C9000089D2C431C600401640F002C10D08400AC
:101CA000A40FA40002AD2C59064D10356219040191
:101CB000650FC401E40EA5401468AC430C431460E6
:101CC00009B0F0BD0002005000ED00E0001BB700BD
:101CD0001C00002080F520000080510100C2EB0BA9
:101CE00000E1F50580F0FA02006A18000024F40013
:101CF000010200002E440000324C080000A24A04F9
:101D000040787D01BC39000053490969382291436C
:101D10000143514A116170474F49096801434E4AD6
:101D2000116070474C49096881434B4A1160704704
:101D30000EB54A4B1A6859689B680293009201914C
:101D4000810F89006A465158434A89184968C30679
:101D5000DB0E01229A401143820F92006B469A5883
:101D60003D4BD21851600EBD0EB53C4B0C331A687A
:101D700059689B68029300920191810F89006A461D
:101D80005158354A89184968C306DB0E01229A402A
:101D90009143820F92006B469A582F4BD218516094
:101DA0000EBD00222E4B1A61042806D11A46126974
:101DB00004231A432A4B1A6106E0274A1269382382
:101DC0009A430243244B1A61254A51610022244B55
:101DD0009A611A46126903231A43214B1A6170470C
:101DE00000201F4908617047FEB5002002901DA029
:101DF000006800901848046A00132040002801D0B1
:101E00000020FEBD0120C0042040002801D0164D56
:101E100000E0164D012040042040002801D0284653
:101E2000EFE7032080032040800B69460A5C0192A3
:101E3000E005C00D861C1F2040022040400A871C80
:101E4000019A7A431146AA087243104600F01AFC20
:101E5000800002900298D4E700020050D4390000BC
:101E600000E000E00102020400805101001BB70005
:101E7000FEB500200290FBA000680090FA48046ABA
:101E800000132040002801D00020FEBD0120C00426
:101E90002040002801D0F54D00E0F54D0120400420
:101EA0002040002801D02846EFE70320800320408F
:101EB000800B69460A5C0192E005C00D861C1F205C
:101EC00040022040400A871C019A7A431146AA0822
:101ED0007243104600F0D6FB800002900298D4E7CF
:101EE000012292020A40002A01D068228261012266
:101EF000D2020A40002A03D0426901231A434261F8
:101F0000012252030A40002A01D0DA4A82610122EA
:101F100092030A40002A01D0426C42640122D2039B
:101F20000A40002A03D08022C261826B826370471C
:101F300000214160704741680322120391434160D0
:101F4000704770B504460D466068A8436060CA4893
:101F5000844203D10C2000F0A2F909E0C748844272
:101F600003D10D2000F09BF902E00C2000F097F95E
:101F700070BD016901225202114301614169521091
:101F800011434161416803221203114341607047CC
:101F900070B504460D46606828436060B6488442C8
:101FA00003D10C2000F074F909E0B448844203D155
:101FB0000D2000F06DF902E00C2000F069F970BD11
:101FC000F0B587B004460D46AD4801460EC9C0685D
:101FD00003AE0EC6069000200290A348406903217C
:101FE00009060840060EA04880690F210902084032
:101FF000070A002020630320E060A068A149084090
:10200000A060012E04D1FFF733FFB10003AA5050A6
:10201000002D26D0B10003AA5058791C00F032FBE5
:10202000690840182946019000F02CFB801E0290A0
:102030009549029888420FD9B10003AA5058791CDB
:1020400000F020FBE90040182946019000F01AFB3F
:102050000009801E606204E003210907029808431A
:10206000606207B0F0BD70B503460C46002111E078
:10207000002506E06D1C01208007854201D3002069
:1020800070BD98690126B60330400028F2D1186867
:102090006054491C9142EBD30846F1E7FFB587B085
:1020A00004460D4617467648103001460EC9C068F2
:1020B00002AE0EC60590002001906B4840690321D6
:1020C00009060840060E684880690F210902084089
:1020D000000A0690012E04D1FFF7CAFEB10002AA41
:1020E0005050002D28D0B10002AA50580699491C22
:1020F00000F0C8FA690840182946009000F0C2FABA
:10210000801E019060490198884210D9B10002AA4E
:1021100050580699491C00F0B5FAE90040182946C4
:10212000009000F0AFFA0009801E606204E0032115
:10213000090701980843606238460A9908431099D4
:102140000843E0600BB0F0BD026A120A12020A43B3
:10215000026242680123DB021A4342607047F7B50E
:1021600086B004460E464648203001460EC9C06877
:1021700001AD0EC50490022020633B484069032155
:1021800009060840070E384880690F2109020840F7
:10219000000A0590012F04D1FFF76AFEB90001AAD9
:1021A0005050002E12D0B90001AA50580599491C70
:1021B00000F068FAF10040183146009000F062FA31
:1021C0000009851E3048854200D2656208980028C3
:1021D00008D1A06A40210843A062A06A0221884376
:1021E000A06207E0A06A20218843A062A06A0221C1
:1021F0000843A06209B0F0BD10B503230363C36AAE
:10220000224C2340C362C36A14060C432343C362B7
:1022100010BD10B501230363C36ACF24A343C36277
:10222000C36A0C4614432343C36210BD70B5034612
:102230000C46002111E0002506E06D1C01208007FE
:10224000854201D3002070BD9869012636073040D1
:102250000028F2D0605C1860491C9142EBD108461E
:10226000F1E7000001020204000200500080510169
:10227000001BB700010000010000054000001540F0
:10228000EC3900000FFFF0FFFFFF0000FFF8FF0038
:10229000C206D20E01219140054A11607047C20664
:1022A000D20E01219140024A803211607047000035
:1022B00000E100E030B589B005462022824901A83E
:1022C00000F00AFA8148854206D181484069072119
:1022D00009020840040A19E07E48854206D17C487C
:1022E0004069072109030840040B0FE07A48854242
:1022F00006D177484069072109040840040C05E02D
:1023000073484069072109050840040D022C03D1D8
:102310007248006809B030BDA00001A90858F9E76B
:10232000F7B582B0064617463046FFF7C3FF019067
:102330000024002501984008B84201D202240CE094
:102340003946019800F09EF90446250E002D04D070
:10235000691C204600F096F9044603982843306033
:102360007460681C60430146019800F08BF905B069
:10237000F0BD0021016041617047FEB505460C4685
:102380002846FFF797FF074600200290394653483A
:10239000006800F077F9401C019000202860686117
:1023A0004F48874209D87D20C000844200D20446AD
:1023B0004B48844208D9044606E0642C00D26424C9
:1023C0004748844200D90446454887420FD8002038
:1023D00002903946434800F055F900907D21C9002C
:1023E00061430846009900F04DF9064610E03C496B
:1023F000384600F047F906466643300E02900298D0
:10240000002805D00299491C304600F03BF90646E9
:102410006E600121890702980843286003E000BF2D
:102420000198401E019001980028F8D100BF28684B
:102430000121490608400028F9D1FEBD10B54369C5
:10244000294C23400B43134308242343436110BD0D
:102450004169082291434161704742695208520024
:102460000A434261026801231B061A430260704757
:1024700001680122120691430160704730B50C4695
:10248000124DA84201D1134D00E0184D2946184DB8
:102490004D60002B01D0202500E000254D61154D39
:1024A000056030BD01680122D2049143016070478C
:1024B000C269520852000A43C2617047C2691623BA
:1024C0009A430A43C26170471C3A00000000014071
:1024D0000002005000010140000011401C000020DB
:1024E00040420F0000CA9A3BEF8FFFFF00011140EE
:1024F000FFFFFF000000084070B5034600200FE01A
:10250000012484400C40002C09D01C68460003259F
:10251000B540AC4346001546B5402C431C60401CFA
:102520001028EDD370BD10B58469130E8B401C4389
:102530008461C3691402240A8C402343C36110BD23
:10254000826901238B409A438261C369024A8A40AF
:102550009343C361704700000100010070B58C0017
:1025600004593425AC4315461D43012635432C43FD
:102570008D00445170BD8A008258520852008B0071
:10258000C250704770B52F48006945076D0F00F0C5
:1025900020F82D490860022D03D0A8002B490C58C3
:1025A00001E029480468274880690007000F461C9D
:1025B0003146204600F066F8254908602549244840
:1025C00000684A10801800F05DF82349086070BD6B
:1025D0007047FEB50020029020A0006800901948C6
:1025E000046A00132040002801D00020FEBD012015
:1025F000C0042040002801D0194D00E0194D0120F1
:1026000040042040002801D02846EFE70320800343
:102610002040800B69460A5C0192E005C00D861CD3
:102620001F2040022040400A871C019A7A4311462D
:10263000AA087243104600F025F880000290029824
:10264000D4E7000000020050240000203C3A0000C3
:102650001C00002040420F00200000200102020464
:1026600000805101001BB700044880470448004720
:10267000FEE7FEE7FEE7FEE7FEE7FEE7D125000006
:10268000C100000030B50B46014600202022012485
:1026900009E00D46D5409D4205D31D469540491B96
:1026A0002546954040191546521E002DF1DC30BDDF
:1026B00070B500242546002801DA01244042002993
:1026C00001DA01254942FFF7DDFFAC4200D040426C
:1026D000002C00D0494270BD03460B439B0703D03A
:1026E00009E008C9121F08C0042AFAD203E00B78D7
:1026F0000370401C491C521EF9D27047F0B51FB43C
:102700000646002082B005464024019100901BE05F
:10271000019922460F46304600F008FA049A059BBC
:10272000801A994110D310461946224600F0EEF95E
:10273000361A8F410197224601200021009F00F0A8
:10274000E5F938184D4100902046641E0028DFDC72
:10275000019B00982946324607B0F0BDF0B5074608
:102760000846584087B0C00F049048000E465900F4
:1027700040084908BC1A884105D2384631461E46F1
:1027800017460B4602465800400810434CD0300D07
:10279000039040055900400D490D0590401A0290E4
:1027A000402872DA18030121000B09050843019043
:1027B00004980092002805D00199524200208841D7
:1027C00000920190029840210A1A0199009800F0A5
:1027D0009DF905460C466B4607CB00F0B8F9C019C9
:1027E0007141039A0E0D0023D71756401A467A40BE
:1027F000164344D0049A002A2DD0029A012A039A43
:1028000015DC1205C01A914101263605001C7141E4
:10281000D20F059ED2070093019202962A462346C4
:1028200000F0B5F907B0F0BD38463146FAE71605B5
:10283000224A0F46B218C01AB74101210905001CEF
:102840004F4100187F41114618187941E20F10439B
:102850006D19644113E0E2076D0815436408C2076F
:102860001443039A01261205C01A91413605001C33
:102870007141CE07400830434908C01851412A46EB
:10288000234600F077F9CDE7FFE7049801224000E6
:10289000C117121A00238B4104983146C417381A05
:1028A000A141EEE730B40124E407634030BC55E7B2
:1028B00030B40124E407614030BC4FE70000E0FF82
:1028C000F0B51FB488B00B990998002448400999C5
:1028D000C00F490049080991C0070B9900904900B1
:1028E00049080B9109990898A64608431CD00B99F2
:1028F0000A98084318D0099801244000420D480066
:10290000410D099824050003000B204309900B9802
:102910000003000B20430B9050181C494018002264
:1029200001901446104605E0002001460DB0F0BDB0
:10293000032801DA034600E003239C46C11A0AAECD
:102940000AE05F0008ADED5B4F00F75B7D430027B9
:10295000AA187C41491C5B1E6145F2DD410004ABB5
:102960005A522104120C0A43240C401C0828DFDBB5
:10297000019802900099704601910090059B049A7D
:102980000799069800F003F9D0E700000DFCFFFF5F
:10299000F0B50C465C4085B0E40FE40703944C00AE
:1029A00000266408590094464908024602962243CC
:1029B00021D062460A431ED06200570D4A000E0322
:1029C0002303550D012402462C492405781B1B0BBB
:1029D000360B401823432643614600901C46501A8C
:1029E000B44103D30098401C009002E09218009874
:1029F0005B41002803DA0020014605B0F0BD00204D
:102A0000012109050746864611E064461D46141B50
:102A1000B54106D36546521BB341744607430C4388
:102A2000A646CD0740084908284392185B41054651
:102A30000D43EAD11046184313D060461946504062
:102A40007140084306D06046101AB34106D20122F5
:102A5000002306E000220123DB0702E00122D2432B
:102A60005310009874460105381C6141029C039D77
:102A70000019694100F07EF8BFE70000FD03000087
:102A80004A0009030123090B1B0519430A4B10B522
:102A9000520D9A4202DA0020014610BD064B343333
:102AA0009A4203DC9A1A00F041F810BD034BD21889
:102AB00000F02CF810BD0000FF030000CDFBFFFF6D
:102AC00010B5002904DB0124E40740428C41214673
:102AD000002B04DB1C460123DB075242A341994231
:102AE00000D1904210BD0000064C0125064E05E0C5
:102AF000E36807CC2B430C3C98471034B442F7D31F
:102B0000FDF7E2FA803A0000A03A000010B5202A52
:102B100004DB0146203A9140002010BD9140202363
:102B20009C1A0346E3401943904010BD10B5202A7B
:102B300004DB0846203AD040002110BD0B46D340AC
:102B4000D0402024A21A91400843194610BD10B568
:102B5000202A06DBCB170846203A1041C1170B4349
:102B600006E00B461341D0402024A21A91400843AE
:102B7000194610BD10B5002B08DA0024401C614135
:102B800092185B411A4301D14008400010BDF0B5D6
:102B90001FB482B005460C0003D0084600F048FA86
:102BA00002E000F045FA2030024600902146284617
:102BB000FFF7ACFF049B059A04460F4618431143E8
:102BC000084314D0184610431BD0009840210A1A1D
:102BD00018460599FFF7AAFF05460E46009A059983
:102BE0000498FFF793FF084305D0012004E0204636
:102BF000394607B0F0BD0020C11705430E432C43F2
:102C0000374300990E986305401A7905E40A0022BB
:102C10000C43FD0A0A3002D500200146E9E7010510
:102C2000101969410C9C0D9D00196941FFF7A2FF25
:102C3000DFE7000010B500BF7C488068C007C00F08
:102C4000002830D000BF01207849886000BF784854
:102C50000068401C76490860322807D300200860CD
:102C60007449C86373494039486205E001207149DD
:102C7000C8637049403948626F48006800281DD019
:102C80006C48006900280BD06A484069002807D0CA
:102C900068488069002803D06648C069002803D1CD
:102CA000142066490860C0E064480068401E63491B
:102CB00008600028F7D160490860B6E05D48006907
:102CC000002813D101205C49086014205B4908608A
:102CD0005B48006864305A490860084600685949F2
:102CE0008842E0DD0846564908609EE05148406948
:102CF000002811D101205049086014204F49086074
:102D00004F48006864384E490860084600686428E7
:102D1000C9DA6420086088E046488069002840D10C
:102D2000012045490860142044490860464800686D
:102D300043490968401A4449086008460068434905
:102D4000884203DA0846404908600CE040480068C1
:102D5000401E3F490860302801DA392008603C49AC
:102D60000878FDF7EBFD38490C68E10F09194910A7
:102D7000384A881834490968FFF784FC401E2C49FA
:102D80000860084601680020FDF72CFC284801680F
:102D90000220FDF727FC264801680420FDF722FCED
:102DA00043E02448C06900283FD10120224908603F
:102DB0001420224908602448006821490968401805
:102DC00021490860084600682349884203DD084617
:102DD0001D4908600CE01E480068401C1C49086042
:102DE000392801DD3020086019490878FDF7A6FD73
:102DF00015490C68E10F09194910164A881812493B
:102E00000968FFF73FFC401E094908600846016851
:102E10000020FDF7E7FB064801680220FDF7E2FB12
:102E2000034801680420FDF7DDFB10BD00010140EF
:102E30002C000020C042005030000020280000205C
:102E4000040000201027000000000020409C00002B
:102E50000800002000A24A04F04902007CB569463F
:102E600001A8FDF70AFE0546002D7DD0642D66D031
:102E70000CDC542D79D004DC202D77D0462D19D1CF
:102E8000A7E0562D73D0612DF9D114E0762D6FD0C7
:102E900004DC662D07D0742DF1D198E0772D39D060
:102EA000782DECD180E04F4802684F4801684F48C8
:102EB000FDF7BEFD94E04C4800684A490968401A95
:102EC00049490860084600684949884202DA0846CC
:102ED0004549086044490E68F10F89194910454A6F
:102EE000881841490968FFF7CDFB441E21460020A0
:102EF000FDF778FB21460220FDF774FB21460420F4
:102F0000FDF770FB37480268374801683748FDF71E
:102F10008FFD65E033480068643032490860084638
:102F200000683549884202DD08462E4908602D4870
:102F300002682D4801682D48FDF77AFD50E02A48C7
:102F40000068284909684018274908600846006851
:102F50002A49884202DD08462349086022490E6852
:102F6000F10F8919491004E03BE033E034E032E02E
:102F70002EE0204A88181C490968FFF783FB441E8D
:102F800021460020FDF72EFB21460220FDF72AFBFB
:102F900021460420FDF726FB12480268124801680A
:102FA0001248FDF745FD1BE00E48006864380D49E6
:102FB000086008460068642801DA6420086009484F
:102FC0000268094801680948FDF732FD08E000BFC2
:102FD00000BF00BF00BF00BF0948FDF729FD00BFCB
:102FE00000BF7CBD04000020000000205C3A00000F
:102FF000409C000000A24A0410270000F049020093
:103000007B3A00007CB51546024600201C4600298C
:103010000BD0491E00920191044B6A462146284676
:1030200000F0F4F8009A002111707CBD45390000D1
:103030002021020C01D010211046020A01D01046B6
:103040000839020901D01046091F820801D0104634
:10305000891E420801D0881E7047081A704730B494
:103060007446641E2578641CAB4204D3635D5B0028
:10307000E31830BC18471D46F8E702E008C8121FE5
:1030800008C1002AFAD170477047002001E001C151
:10309000121F002AFBD17047F0B51FB486B0099803
:1030A000089A030D0021024314D05148514A1818C0
:1030B000504305141198012810981AD0281A401C62
:1030C00000264D4F4D49009601910490002812DAD8
:1030D000444211E01198012449A3012801D110981C
:1030E000C1430698119A84600360C26041600BB0CE
:1030F000F0BD4042E4E70446210500203F4A001CA1
:1031000051410391029012E0E00707D032463B465E
:1031100001990098FFF7D4FB0191009032463B469D
:1031200010461946FFF7CCFB06460F466410002CEC
:10313000EAD10498039B0028029A0999089806DAB4
:10314000FFF7BEFB019B009AFFF7BAFB05E0FFF714
:103150001FFC019B009AFFF71BFC04460E46002251
:10316000284BFFF7ADFC03D80020C043014607E021
:103170000022254B20463146FFF7F0FAFFF780FC8E
:10318000102409E0002C0ADB0A220023FFF7B6FA1C
:10319000079B30321A55641E02460A43F2D11122AF
:1031A000641C079B121B1C19119B012B03D00123CC
:1031B00008430ED10AE0084304D0112010900020EB
:1031C000119077E71098151A6D1E0BE01098824247
:1031D00002DD00236D1C03E0824201DA00236D1E34
:1031E000002BEED0069811998260C16030C07EE756
:1031F00001FCFFFF104D0000000014400000F03FF4
:10320000300000000000F0430000E03FFFB597B041
:103210000646002518E2252877D100242746FD49D7
:10322000049400E00443761C32780120203A904058
:103230000842F7D130782A280ED002223078014691
:103240003039092916D804990A23594330394018CE
:103250001443761C0490F1E7189802C80491189062
:10326000002904DA0120400304434842049002206C
:103270000443761C30782E2814D10420044370783F
:10328000761C2A2809D11898761C80C8189009E065
:103290000A214F43303FC719761C30780146303938
:1032A0000929F5D930786C2810D006DC4C281AD0C2
:1032B00068280ED06A2817D104E0742813D07A2821
:1032C00012D110E00120400504430CE00121090562
:1032D00001E0032109050C437178814203D10120EB
:1032E00000052418761C761C3078119066280BD0C7
:1032F00013DC58287DD009DC00287BD04528F6D087
:103300004628F4D047281AD1A5E118E0632835D023
:10331000642870D0652812D19DE170286CD008DC3B
:103320006728F1D069287BD06E280DD06F2806D190
:10333000BAE073282ED0752871D0782859D01A9AFF
:10334000199990476D1C7EE16002400F022809D058
:1033500003280DD00428189801680DD00D60001DB9
:10336000189070E11898EA1701680D604A60F6E756
:10337000189801680D80F2E70D70F0E718986A461A
:1033800001781172001D18900020507202A8009060
:10339000012005E0189802C8189000200091C04351
:1033A00061070DD5002101E00199491C0191B94245
:1033B00012DA8142F8DB009A515C0029F4D10BE06B
:1033C000002101E00199491C01918142FADB019A37
:1033D0000099895C0029F5D1019904981A9B471A34
:1033E00021463846199A00F097FA01994019451874
:1033F0000BE04FE02CE113E04EE0009800990078DC
:10340000491C00911A9A199990470198401E019001
:10341000401CF2D1214638461A9B199A10E137E038
:103420000A200021009001916002410F022907D07B
:10343000189A01CA1892C2179446032908D00AE0C4
:103440001898C01DC108C90005C91891944607E025
:1034500000B2C2179446042902D140B2C1178C466B
:1034600000226146944506DA0A4600214042914115
:103470008C462D2102E0210504D52B216A461173CB
:10348000012103E0E10701D02021F7E7029155E097
:103490000A200AE0102008E01020009000210420FB
:1034A00004430191082703E00820002101910090C6
:1034B0006002410F022907D0189A01CA189200220F
:1034C0009446032908D008E01898C01DC108C90017
:1034D00005C91891944603E080B2042900D1C0B216
:1034E00000210291210729D51199702906D0009A4F
:1034F0001021019B4A401A4305D00EE040216A4644
:103500001173012108E06146014306D030216A466B
:1035100011731199517302210291009A0821019BA4
:103520004A401A430AD16146014301D1610705D5DA
:1035300030216A46117301217F1E02911199582989
:1035400004D035A10E910DA90D910DE037A1F9E739
:103550006146019B009AFFF7D1F80E9B8C469B5C5D
:103560000D9A521E0D92137061460143F0D10D98D1
:1035700005A9081A20300190600703D50120000436
:10358000844300E001270198874201DD381A00E0FA
:103590000020019900904118029809180498401AD7
:1035A0000490E00306D421461A9B199A049800F06F
:1035B000B3F94519002706E003A81A9AC05D1999C6
:1035C00090476D1C7F1C02988742F5DBE0030CD509
:1035D00021461A9B199A049800F09EF9451904E0B7
:1035E0001A9A3020199990476D1C0099481E009036
:1035F0000029F5DC08E00D980D990078491C0D9123
:103600001A9A199990476D1C0199481E019000293A
:10361000F1DC63E1092801003031323334353637CB
:10362000383961626364656600000000303132330E
:1036300034353637383941424344454600000000AE
:1036400000F05AF94519761C3078002800D0E2E5E0
:1036500028461BB0F0BD600700D406271898C01D8F
:10366000C108C90048680A680831C30FDB07189110
:10367000190001D09CA108E0210501D59BA104E01F
:10368000E10701D09AA100E09AA1430011985B08DC
:10369000109165280CD006DC452809D046281DD09D
:1036A000472841D141E0662818D067283CD13CE04A
:1036B0000021112F01DB112000E0781C0191009006
:1036C00008A911A8FFF7E8FC139905910021119AA8
:1036D00015927F1C12980197009150E00120C007BD
:1036E00003900120019008A9009711A8FFF7D4FCCE
:1036F000139A149905920022119B00921298159327
:10370000059A0192002901D0104602E0791C401868
:103710000190381A01D5019804E04042401E009003
:10372000781C0190C01B029043E0012F00DA0127B2
:103730000021112F01DD112000E038460191009099
:1037400008A911A8FFF7A8FC13990591119A002167
:10375000129815920091019721070CD40599B9424E
:1037600001DB019900E00191012904DD159A491E50
:10377000515C302906D0B84201DA011D05DA012179
:10378000029115E00199491EEDE7002805DC00993A
:10379000411800910199091A03E0019A411C9142D4
:1037A00000DD01910099401A401C02900120C007E1
:1037B0000390200706D402990198814202DB002081
:1037C000C043029000206946C87707AF01210398E3
:1037D0000337C907884224D0022011902B20129071
:1037E000039800280CDA404203902D20129007E045
:1037F0000A210398FEF746FF30317F1E039039708F
:103800001199481E11900029F2DC03980028EFD18D
:10381000791E129808703078202108404530BF1E6C
:10382000387006A8C01BC01D0390109800780028AF
:1038300000D00120019941180298C0170918039877
:1038400009180498401A401E0490E00306D421464B
:103850001A9B199A049800F05FF84519109800789F
:10386000002803D01A9A199990476D1CE00324D5BB
:1038700021461A9B199A049800F04EF845191CE04D
:103880000098002807DB00990598884203DD159809
:10389000405C199901E0199930201A9A90470098D4
:1038A0006D1C401C00900298401E0290002804D11C
:1038B0001A9A2E20199990476D1C0199481E019063
:1038C0000029DDDC05E038781A9A7F1C19999047A9
:1038D0006D1C0399481E03900029F4DC21461A9BB5
:1038E000199A0498ACE600002D0000002B0000009F
:1038F0002000000000000000F8B5044600251E4628
:103900001746880404D405E039462020B0476D1CD2
:10391000641EF9D52846F8BDFFB50446002581B0E0
:103920001E46C80301D5302700E02027880404D5AF
:1039300005E038460399B0476D1C641EF9D528464A
:1039400005B0F0BD4A68002A06D00A68531C0B6017
:1039500010704868401E48607047003022416D5228
:103960007C20390F2170084080523F065B4F666D06
:103970007D077F6F484839480F535F777C395E7900
:10398000713D76061E763815373F7367316D786E58
:103990001C2A766E5B39640F230820777C585E7989
:1039A000716F74041E761815545C7667506D783EFE
:1039B0001C2A76675B466E3D6D6E6E00000000004F
:1039C000040000000C0000002400000000000000C3
:1039D0002000000000000000040000002C00000097
:1039E00000000000040000002C000000001BB700D5
:1039F000000000000080000000805101001BB700A3
:103A0000000000000080000000805101001BB70092
:103A1000000000000080000000805101001BB70082
:103A20000080000000000000000000000000000016
:103A3000102700000000000000805101001BB700AB
:103A40000080000000E0480410270000006CDC0249
:103A500000000000000000000080510143757272F8
:103A600046726571203D2025642044656C74614672
:103A7000726571203D2025640D0A004E410D0A003B
:103A8000A03A000000000020340000007A3000005E
:103A9000D43A000034000020040400008A30000002
:103AA000F049020010270000300000000000000074
:103AB00000000000000000000000000000E04804DA
:103AC0004700000000E04804000000000000000083
:043AD00000000000F2
:040000050000266968
:00000001FF
